:100000000C945A000C9477000C9477000C947700B1
:100010000C9477000C9477000C9477000C94770084
:100020000C9477000C9477000C9477000C94770074
:100030000C9477000C9477000C9477000C94770064
:100040000C9493010C9477000C9477000C94770037
:100050000C9477000C9477000C9477000C94770044
:100060000C9477000C947700000024272A000025C8
:10007000282B000023262904040404040404040299
:100080000202020202030303030303010204081035
:100090002040800102040810200102040810200002
:1000A0000000070002010000030406000000000039
:1000B0000000000011241FBECFEFD4E0DEBFCDBF93
:1000C00011E0A0E0B1E0EEE4F6E002C005900D9290
:1000D000AE30B107D9F711E0AEE0B1E001C01D923A
:1000E000A831B107E1F70E948C010C9425030C9410
:1000F000000061E0809100010E9470020895BF92AB
:10010000CF92DF92EF92FF920F931F93DF93CF93E3
:10011000CDB7DEB72A970FB6F894DEBF0FBECDBFBE
:100120006B01DE011196E4E0F1E02AE001900D920E
:100130002150E1F79C0189589F4FFC01849125577C
:100140003F4FF901B490E82FF0E0EE0FFF1FEC0FE6
:10015000FD1F0181128190E2E92EF12CE00EF11ECB
:10016000F80180A18B2980A38AE090E00E942802F8
:10017000F894F80180A19B2D9095892380A300001D
:10018000000000000000000000000000000000006F
:10019000000000000000000000000000000000005F
:1001A000000000000000000000000000000000004F
:1001B000000000000000000000000000000000003F
:1001C000000000000000000000000000000000002F
:1001D000000000000000000000000000000020E01F
:1001E00030E0C0FE04C0F70180818B2903C0F70115
:1001F000808189238083000000000000000000004F
:1002000000000000000000000000000000000000EE
:1002100000000000000000000000000000000000DE
:1002200000000000000000000000000000000000CE
:1002300000000000000000000000000000000000BE
:1002400000000000000000000000000000000000AE
:100250000000000000002F5F3F4F2830310519F0EB
:10026000D594C794BECFF80180A18B2980A3789440
:100270002A960FB6F894DEBF0FBECDBFCF91DF91A7
:100280001F910F91FF90EF90DF90CF90BF90089556
:10029000CF93DF9360E0809100010E948E026AE0BC
:1002A00070E080E090E00E94FE0160E070E08091EC
:1002B0000001909101010E947F00C1E0D0E06091B7
:1002C0000E0170910F0180910001909101010E9437
:1002D0007F00219682E0C130D80789F72091020182
:1002E0003091030180910E0190910F01820F931FB5
:1002F00090930F0180930E01009719F08F3F9105A5
:1003000041F488279927821B930B909303018093D4
:100310000201DF91CF9108950E9436020E94790078
:100320000E944801FDCF1F920F920FB60F92112429
:100330002F938F939F93AF93BF93809110019091D0
:100340001101A0911201B09113018050904CAF4F58
:10035000BF4F8093100190931101A0931201B093AD
:10036000130127C08091100190911101A0911201F9
:10037000B091130180589E43A040B040809310017B
:1003800090931101A0931201B09313018091140175
:1003900090911501A0911601B09117010196A11D30
:1003A000B11D8093140190931501A0931601B09391
:1003B00017018091100190911101A0911201B0914B
:1003C000130181589E43A040B04060F6BF91AF91A9
:1003D0009F918F912F910F900FBE0F901F901895A6
:1003E0008FB7F894209114013091150140911601B6
:1003F000509117018FBFB901CA010895EF92FF9282
:100400000F931F937B018C018FB7F89440911401D7
:100410005091150160911601709117018FBF2FB790
:10042000F8948091140190911501A0911601B0915A
:1004300017012FBF841B950BA60BB70B8E159F05BD
:10044000A007B10760F31F910F91FF90EF900895FF
:10045000019759F0FC01EE0FFF1FEE0FFF1F3297BF
:100460008FB7F8943197F1F78FBF0895789484B5DA
:10047000826084BD84B5816084BD85B5826085BDA0
:1004800085B5816085BDEEE6F0E080818160808386
:10049000E1E8F0E0808182608083808181608083F8
:1004A000E0E8F0E0808181608083E1EBF0E0808132
:1004B00084608083E0EBF0E0808181608083EAE704
:1004C000F0E080818460808380818260808380818D
:1004D000816080838081806880831092C10008954C
:1004E000282F30E0C90185579F4FFC01949129586E
:1004F0003F4FF9018491882381F0E82FF0E0E8591B
:10050000FF4FE491F0E0662329F4808190958923E0
:10051000808308958081892B80830895482F50E03F
:10052000CA0181569F4FFC012491CA0185579F4FF4
:10053000FC01949149585F4FFA0134913323C1F182
:10054000222331F1233021F4809180008F7705C080
:10055000243031F4809180008F7D8093800018C01A
:10056000213019F484B58F7704C0223021F484B58A
:100570008F7D84BD0DC0263021F48091B0008F772F
:1005800005C0273029F48091B0008F7D8093B000A2
:10059000E32FF0E0E359FF4FE491F0E0662329F404
:1005A000808190958923808308958081892B808321
:1005B0000895482F50E0CA0181569F4FFC012491B5
:1005C000CA0185579F4FFC01949149585F4FFA012A
:1005D0003491332319F420E030E035C0222331F187
:1005E000233021F4809180008F7705C0243031F4CE
:1005F000809180008F7D8093800018C0213019F495
:1006000084B58F7704C0223021F484B58F7D84BDFA
:100610000DC0263021F48091B0008F7705C02730BF
:1006200029F48091B0008F7D8093B000E32FF0E03B
:10063000EE58FF4FE491F0E0808120E030E0892324
:0E06400011F021E030E0C9010895F894FFCFD9
:0E064E000800030000000000050008000B007B
:00000001FF
